:03000000023A6061
:0C3A600078FFE4F6D8FD758171023AA7EA
:100F980020000A3C2E2E2E3E004950436F6E6E658F
:100FA80063745245510A004950436F6E6E6563740D
:100FB800000A49504E6F41434B210A003E432C56CC
:100FC8002C43432CC0E4E0EFF2E5F020D1E8EDEA51
:100FD800EEEC49500A003E432C4D41432C2530325B
:100FE80062583A25303262583A25303262583A25EA
:100FF800303262583A25303262583A2530326258D7
:101008002C4D414320E0E4F0E5F10A003E432C5624
:1010180045522C20332E3220EEF2202573202573E2
:101028002CC2E5F0F1E8FF20495020ECEEE4F3EBA8
:10103800FF0A0044656320313420323031300031FA
:10104800343A32383A3239003E432C4C442C505210
:101058004F473A2020202020202020202020202018
:101068002020202020202020202020202020202078
:101078002020202020202020202020202020202068
:101088002020202020202020202020202020202058
:1010980020202020202020202CC4E0F2E020EFF0A7
:1010A800EEF8E8E2EAE828F4E0E9EB290A003E2A4B
:1010B8002C312CCEF1EDEEE2EDFBE520EFE0F0E097
:1010C800ECE5F2F0FB20F1E5F2E5E2EEE3EE20E8F4
:1010D800EDF2E5F0F4E5E9F1E00A003E412C41309B
:1010E800312C2562752E2562752E2562752E256296
:1010F800752C495020E0E4F0E5F120E0E4E0EFF25F
:10110800E5F0E00A003E412C4130322C2562752E74
:101118002562752E2562752E2562752C495020E0B2
:10112800E4F0E5F120EEF1ED2E20F1E5F0E2E5F056
:10113800E00A003E412C4130332C2562752E256291
:10114800752E2562752E2562752C495020E0E4F035
:10115800E5F120F0E5E72E20F1E5F0E2E5F0E00A20
:10116800003E412C4130342C2562752E2562752EA7
:101178002562752E2562752CCCE0F1EAE020F1E5B8
:10118800F2E80A003E412C4130352C2562752E25A7
:1011980062752E2562752E2562752CD8EBFEE70A3E
:1011A800003E2A2C312CC4EEEF2E20EFE0F0E0ECCC
:1011B800E5F2F0FB20F1E5F2E5E2EEE3EE20E8ED02
:1011C800F2E5F0F4E5E9F1E00A003E422C53303153
:1011D8002C2562752CC6E4E0F2FC20E7E0EFF0EE87
:1011E800F1E020F1EEE5E4E8EDE5EDE8FF20EEF2D0
:1011F80020F1E5F0E2E5F0E00A003E422C533032FF
:101208002C2562752CCEE1ECE5ED20F120F1E5F01E
:10121800E2E5F0EEEC20E1E5E720EAE2E8F2E0EDD5
:10122800F6E8E90A003E422C5330332C2562752C2F
:10123800CFE5F0E5E7E0EFF3F1EA20EFF0E820EFA3
:10124800EEF2E5F0E520F1E2FFE7E820F120F1E534
:10125800F0E2E5F0EEEC0A003E422C5330382C2543
:1012680062752CCCE5E4EBE5EDEDFBE92049502077
:10127800EAE0EDE0EB28E7E0E4E5F0E6EAE020E488
:10128800EE203520F1E5EA290A003E422C5330359C
:101298002C2562752CCAE0EDE0EB20F8E8F0EEEAC8
:1012A800EEE2E5F8E0F2E5EBFCEDEEE3EE20EEE150
:1012B800ECE5EDE00A003E532C5330362C25303255
:1012C80062582530326258253032625825303262F1
:1012D80058253032625825303262582C4D4143200F
:1012E800E0E4F0E5F120F8E8F0EEEAEEE2E5F8E017
:1012F800F2E5EBFCEDEEE3EE20EEE1ECE5EDE00AE5
:10130800003E454E440A000A44756D70582020205E
:10131800202030302030312030322030332030341B
:1013280020303520303620303720303820303920F2
:101338003041203042203043203044203045203096
:1013480046000A3A003A20000A000A44756D7044C3
:1013580020202020203030203031203032203033FF
:1013680020303420303520303620303720303820B7
:101378003039203041203042203043203044203062
:101388004520304600457272206B65790052642012
:10139800656570726F6D0A005264204D454D0A00F4
:1013A800526420436F64650A00577269746520436C
:1013B8006F64650A0044656275674950204F4E0A9C
:1013C8000044656275674950204F46460A004465E7
:1013D80062756755736572204F6E0A0044656275C1
:1013E8006755736572204F46460A00446562756703
:1013F8004D7367204F6E0A0044656275674D7367C9
:10140800204F46460A00436F6E666967206C6F631B
:101418006B210A00577220656570726F6D0A002093
:101428005361766520656570726F6D210A0045729B
:1014380072204D414321004C6F61643E3E002A00FA
:10144800CEF8E8E1EAE00A00202D20257528257568
:10145800290A003C4130313D003C4130323D003CDE
:101468004130333D003C4130343D003C4130353D56
:10147800003C21003C5330313D003C5330323D00AC
:101488003C5330333D003C5330353D003C533038FD
:081498003D003C5330363D00DD
:06447A00010B0001090026
:10443D00C28E438910758BFF758DB7D2ABD28E228C
:03001B000239D0D7
:1039D000C0E0C083C082C0D0C28E758BFF758DB72A
:1039E00020060675A61E75A6E10509D202E50B6044
:1039F00002050B050EE50E540F7051E50AD3940134
:103A00004002150AD20EE50E543F7012D200907794
:103A100059E0600A04F0E0D394B44002D2069077F3
:103A200052E0600204F09071CFE0600214F09077F1
:103A30005AE0D394014003E014F0300502050CE590
:103A40000DD394644004D2068002050DE508D3949A
:103A50000140021508D28ED0D0D082D083D0E0327F
:10091100C291C290D2B5C20B7D027C007F07124406
:10092100068F25E525646060097D017F601243A182
:10093100D20BE4FDFC7F0B1244068F25E52530E642
:10094100097D04E4FF1243C5D20B7D017C007F07C2
:100951001244068F25E5257008FD7FFF1243A1D2C1
:100961000B300B03126000C288C2A8C2AA758900AD
:10097100123E0C90740AE0B4FA06A3E064CE607BE8
:10098100E4F52574022525F582E43474F583E4F059
:100991000525E525B443EC90740A74FAF0A374CEEE
:1009A100F0A374CCF0907410740AF0E4A3F0A304E3
:1009B100F0A3F090740674FFF0A3F0A3F0E4A3F0A9
:1009C1009074217403F0E4F525E5252401FFE43357
:1009D100FE74022525F582E43474F583E0FD1243AB
:1009E1007D0525E525C3944340DFE4F5A775A61EE3
:1009F10075A6E1907FF0F0A3F080FE90741574036A
:100A0100F0A374CCF0E4907414F0907757F0A3F055
:100A11001233DBC2B51237DCC2061240EED20BC272
:100A21000DC20C9076427408F09073807424F0E447
:100A3100A3F090740AE0907382F090740BE09073CD
:100A410083F090740CE0907384F090740DE09073D7
:100A510085F090740EE0907386F090740FE09073BF
:100A610087F0750A01E4907643F0C207C208C20913
:100A7100C20A124356200B19AF257E007D031234A2
:100A8100C1E4FF12372C7E0F7F98E4FBFDFC122F8F
:100A9100FF907759E060037401F0E49071CFF0F5B5
:100AA1000C907641F0F50D12443D75A70775A61E11
:100AB10075A6E1D2AFE4F50D9071CFE07003121C81
:100AC1007390775AE06401701D9080007410F0906B
:100AD10080A874FFF0A3F0A3F0A3F0E490775AF09C
:100AE100D20BC20CC20D908008E0F52530E405D28E
:100AF100077410F0E52530E508D2099080087420CC
:100B0100F0E52530E608D2089080087440F0E50C45
:100B1100C394034019908002E4F0908001F090802A
:100B210000F0E50C94064006E4F50C1240EE9080CE
:100B3100A0E07003123F049080B8E07003123E8A77
:100B41009080D0E07003124092908000E0701330EA
:100B510007101231069073FDEFF0D3940040031299
:100B61000026908002E07006908000E06005D205CA
:100B7100020AB6C205E4F50C9071CFE06003020AE7
:100B8100B6200B12907644E0600C7E0F7F9A1232F1
:100B9100F3E4907644F0300912122C099073FDEFC2
:100BA100F0D394004005E0FF12444D200803020DEC
:100BB1003A122A829073FDEFF07003020AB6907424
:100BC10041E054BF247F7003020C95147003020CA2
:100BD1006D24026003020CDC200B077E0F7FA11243
:100BE10032F3200F03020D3A907419E070069074ED
:100BF1001DE0606790774EE0FF907419E0B507241F
:100C010090774FE0FE90741AE0B50618907750E0A7
:100C1100FE90741BE0B5060C907751E0FE90741CB9
:100C2100E06E603790741DE06F6003020D3A9077BB
:100C31004FE0FF90741EE06F6003020D3A90775011
:100C4100E0FF90741FE06F6003020D3A907751E06E
:100C5100FF907420E06F6003020D3AC20390764367
:100C61007401F0120021750A01020D3A907759E0E2
:100C710060037401F0907746E0FF907443E06F6089
:100C810003020D3A907746E004F0E4F50A907641CC
:100C9100F0020D3A300303020D3A907410E0700334
:100CA100020AB690737FE06008907421741EF08090
:100CB100069074217403F0124481D203E4F50A9082
:100CC1007641F090775204F0E4907745F0A3F0205C
:100CD1000B677E0F7FAF1232F3805E907759E06031
:100CE100037401F0300352907441E020E74B90749B
:100CF10043E0FF907745E0FE6F600D90774DE07027
:100D010007EE146F70338013907745E004F0907311
:100D1100FDE0FFD3940440031242239070CB748210
:100D2100F0A37401F0907443E09070CDF07E707F79
:100D3100CB7D03123B73020AB6200303020E58E572
:100D41000A706E1242CDEF60237E757F419075422D
:100D5100E02404FD123B7390774DE07009907421FB
:100D6100E0F50A020AB6E4F50A020AB6907752E003
:100D7100D3943C403C90774DE0703690737FE070A7
:100D81003090775204F0124467E4907541F0A374F7
:100D910012F0907746E0907543F0A374FDF09071E6
:100DA100D063A20190754563A2017F1212260680CD
:100DB1009812445C8F25E525B401159070CB74839E
:100DC100F0E4A3F07E707FCB7D02123B73020AB682
:100DD100E525D39401401C9070CB7483F0A374017A
:100DE100F0E52524FEA3F07E707FCB7D03123B73DB
:100DF100020AB6E50A64016003020AB6907641E090
:100E010004F0200B077E0F7FB91232F3907421E0BA
:100E1100C3941E5004E02402F0907641E0C394058F
:100E2100400DC203E4907643F0120021020AB67C21
:100E3100777D4E907415E0FAA3E0FB7F02123D042A
:100E41007E757F41907542E02404FD123B739074DE
:100E510021E0F50A020AB6E50A64016003020AB656
:100E6100907643E014604624FE6042147003020F42
:100E71004B24046003020AB6E4F50C200F139076AC
:100E8100437404F0907641E05401F0750A01020ABE
:100E9100B69080027410F0E4907643F090764104AD
:100EA100F0750A1290774E74FFF0020AB690774EF1
:100EB100E07003020F359075417480F090754374B2
:100EC10001F0E4A3F0A304F0A37430F0A3747BF069
:100ED100E4F52574482525F582E43475F583747DA0
:100EE100F074492525F582E43475F583E4F0E525B0
:100EF1002407907542F07C777D4E907415E0FAA33B
:100F0100E0FB7F02123D047E757F41E5252409FD4A
:100F1100123B7390774DE0601B124481D203E4F5DC
:100F21000A907641F090775204F0E4907745F0A36F
:100F3100F0020AB6300F07E4907643F0800690760F
:100F4100437404F0750A12020AB69080027410F01C
:100F5100750A03907641E06401FFF09076437401D5
:100F6100F0EF701990741DE06013FCA3E0FDA3E0A5
:100F7100FEA3E0FF90774E12239B020AB6907419EC
:100F8100E0FCA3E0FDA3E0FEA3E0FF90774E122377
:060F91009B020AB680FE7F
:010F97002237
:10002600907442E0B444047F0180027F00907441E2
:10003600E0B447047E0180027E00EE5F604A907461
:100046000AE0907443F090740BE0907444F090745E
:100056000CE0907445F090740DE0907446F0907446
:100066000EE0907447F090740FE0907448F090742E
:10007600427452F090737963A2019080A863A20142
:100086007F061226060209079073FDE0C394085006
:100096000302091090740AE0FF907443E06F600356
:1000A60002091090740BE0FF907444E06F60030245
:1000B600091090740CE0FF907445E06F600302092C
:1000C6001090740DE0FF907446E06F600302091013
:1000D60090740EE0FF907447E06F60030209109081
:1000E600740FE0FF907448E06F600302091090748B
:1000F60042E06444701A9080A8E0B4FF13907379CC
:1001060063A2019080A863A2017F061226068010D2
:1001160090737DE09080ACF090737EE09080ADF0BF
:10012600907759E060037401F090775A7464F09008
:1001360074427452F0907441E0646D60030202AA46
:100146007BFF7A0F79C41219797BFF7A0F79DE90DB
:10015600740AE0F52EA3E0F52FA3E0F530A3E0F551
:1001660031A3E0F532A3E0F533121979752EFF7548
:100176002F1075303B7531FF7532107533477BFF95
:100186007A1079141219797BFF7A1079501219793D
:100196007BFF7A1079B61219797BFF7A1079E39092
:1001A6007410E0F52EA3E0F52FA3E0F530A3E0F5FB
:1001B600311219797BFF7A11790D907419E0F52EB9
:1001C600A3E0F52FA3E0F530A3E0F5311219797B12
:1001D600FF7A11793B90741DE0F52EA3E0F52FA36D
:1001E600E0F530A3E0F5311219797BFF7A117969D0
:1001F600907406E0F52EA3E0F52FA3E0F530A3E01A
:10020600F5311219797BFF7A11798C907402E0F539
:100216002EA3E0F52FA3E0F530A3E0F5311219790E
:100226007BFF7A1179A91219797BFF7A1179D2A20B
:100236000FE433F52E1219797BFF7A127902907743
:100246004DE0F52E1219797BFF7A12792D907759A8
:10025600E0F52E1219797BFF7A12796090737FE0B0
:10026600F52E1219797BFF7A127992A201E433F501
:100276002E1219797BFF7A1279BE907747E0F52E18
:10028600A3E0F52FA3E0F530A3E0F531A3E0F532C6
:10029600A3E0F53312197912388A7BFF7A137909AC
:1002A60012197922907441E0644C70737E137F0FAB
:1002B600FBFDFC122FFF907449E0F526A3E0F5271D
:1002C600E4F529E52690744BF0A3E527F07E137F2D
:1002D6004A7C747D4B7B02122FFFE4F5288527822A
:1002E600852683E0FF744B2528F582E43474F58374
:1002F600EFF00527E527700205260528E528B41046
:10030600DC7E137F4D7C747D4B7B10122FFF0529FD
:10031600E529C3941040AC7E137F501232F322902D
:100326007441E0646C7060F52A7E137F52FBFDFC1D
:10033600122FFFE4F529E490744BF0A3E52AF07E32
:10034600137F4A7C747D4B7B02122FFFE4F528A8AD
:100356002AE6FF744B2528F582E43474F583EFF022
:10036600052A0528E528B410E67E137F4D7C747DAA
:100376004B7B10122FFF0529E529C3940840B77E51
:10038600137F501232F322907441E0644B7061F592
:100396002874332528F582E43474F583E0603274DA
:1003A600332528F582E43474F583E0F4602374334E
:1003B6002528F582E43474F583E0FF74492528F591
:1003C60082E43474F583E0B507100528E528B408FF
:1003D600C09071CF7432F00209079074417421F015
:1003E600300B030209077E137F8D1232F3020907D1
:1003F600907441E0B4521A200B077E137F95123297
:10040600F39074417472F07E747F417D08123AEC69
:1004160022907441E064497045200B077E137FA04B
:100426001232F3907449E0F526A3E0F527E4F528A7
:10043600852782852683E0FF744B2528F582E434E0
:1004460074F583EFF00527E527700205260528E5F4
:1004560028B480DC7E747F417D8A123AEC22907447
:1004660041E064437046200B077E137FA81232F3E7
:10047600907449E0F526A3E0F527E4F52885278260
:10048600852683E493FF744B2528F582E43474F5BE
:1004960083EFF00527E527700205260528E528B431
:1004A60080DB7E747F417D8A123AEC22907441E0B3
:1004B600645A7053200B077E137FB11232F3907487
:1004C60049E0F526A3E0F5277C747D4B7B80AF27BA
:1004D600AE26124299E4F528852782852683E49381
:1004E600FF744B2528F582E43474F583EFF0052775
:1004F600E527700205260528E528B480DB7E747F93
:10050600417D8A123AEC22907441E0644460030211
:10051600059E907449E0FF64447003020907EFB436
:10052600310CC20B7E137FBD1232F30209079074A1
:1005360049E0B4300CD20B7E137FC91232F30209A4
:1005460007907449E0B4320CD20C7E137FD6123277
:10055600F3020907907449E0B4330CC20C7E137F92
:10056600E41232F3020907907449E0B4340CD20D58
:100576007E137FF31232F3020907907449E0B43513
:100586000CC20D7E147F001232F3020907907449E3
:10059600E0FF12001E0209079071CFE07013200BD6
:1005A600077E147F0E1232F39074417421F0020913
:1005B600079071CF7432F0907441E0FFB45104C2D9
:1005C600AF80FEEF64577045200B077E147F1C1228
:1005D60032F390744AE09073FDF0E4F5289073FDD1
:1005E600E0FFE528C39F4003020907744B2528F561
:1005F60082E43474F583E0FF907449E0252824787A
:10060600F582E43472F583EFF0052880D0907441CA
:10061600E0645360030206C1200B077E147F271295
:1006260032F390740AE0FF907281E06F703C907430
:100636000BE0FF907282E06F703090740CE0FF90D8
:100646007283E0B5072490740DE0FF907284E0B5E4
:10065600071890740EE0FF907285E0B5070C907451
:100666000FE0FF907286E06F60169074417421F07F
:10067600300B030209077E147F361232F302090794
:10068600E4F528E4F50DAF28FE74782528F582E414
:100696003472F583E0FD12437D0528E528C394FEF8
:1006A60040E1C2AFE4907FF0F0A3F0907FFD74AA22
:1006B600F0A374FFF0A37455F080FE907441E064DB
:1006C6004F705A907449E0F526A3E0F527E52745D3
:1006D60026700A200B077E147F3F1232F3200B0789
:1006E6007E147F461232F3E4F528744B2528F582F2
:1006F600E43474F583E0852782852683F00527E5B3
:1007060027700205260528E528B480DE907758E094
:100716002480F0907757E03400F002090790744186
:10072600E064457074907449E0FEA3E0FF907FF0AA
:10073600EEF0A3EFF0D39400EE94044038907FF0EF
:10074600E0FEA3E0FF907757E0FCA3E0FD9FEC9E60
:100756004023E42FFFEE3401FED3ED9FEC9E5015AF
:10076600C2AF907FFD74AAF0A374FFF0A37455F096
:10077600E4F5A780FE7E147F481232F37BFF7A14DD
:100786007950907FF0E0F52EA3E0F52F907757E0B3
:10079600F530A3E0F531121979907441E064656093
:1007A60003020910907449E0FFA3E0907FF0CFF0B8
:1007B600A3EFF0E4F526F527D3907FF1E095279097
:1007C6007FF0E095264020E4F50D2527FFE5263449
:1007D60001FE852782852683E0FD12437D0527E5F8
:1007E600277002052680D17E147F5B123BFAEF4EFE
:1007F6006020120003907410EFF012000390741141
:10080600EFF0120003907412EFF0120003907413CD
:10081600EFF07E147F61123BFAEF4E602012000368
:10082600907419EFF012000390741AEFF01200039F
:1008360090741BEFF012000390741CEFF07E147F8F
:1008460067123BFAEF4E602012000390741DEFF022
:1008560012000390741EEFF012000390741FEFF065
:10086600120003907420EFF07E147F6D123BFAEFB6
:100876004E6020120003907406EFF012000390748D
:1008860007EFF0120003907408EFF0120003907463
:1008960009EFF07E147F73123BFAEF4E60201200D0
:1008A60003907402EFF0120003907403EFF012004D
:1008B60003907404EFF0120003907405EFF0E4F572
:1008C60028E4F50DE5282401FFE433FE740225280B
:1008D600F582E43474F583E0FD12437D0528E528AE
:1008E600C3944340DCC2AFE4907FF0F0A3F0907F66
:1008F600FD74AAF0A374FFF0A37455F0E4F5A78085
:0A090600FE7E747F417D08123AEC7A
:0109100022C4
:10426100AE07EEC39430400BEED394395005EE24E3
:10427100D0FF22EEC39461400BEED394665005EE5D
:1042810024A9FF22EEC39441400BEED3944650057E
:08429100EE24C9FF22AF062252
:10442300907378E004F07006907377E004F0907373
:0A44330077E0FEA3E0FF1243E92248
:10000300124423124261EFC454F0FEC0061244238B
:08001300124261D0E02FFF2230
:10403500E49078B3F01244239078B4EFF0C3943051
:104045004018E0FFD3943950119078B3E024D0F5AF
:1040550082E43471F583EFF080119078B3E024D0D9
:10406500F582E43471F583E4F0800C9078B3E004D4
:10407500F0E0D3940840BE752900752A00752B0021
:0C408500E4F52C7B017A7179D01228DE62
:01409100220C
:043BFA008E2B8F2C53
:103BFE00907377E4F0A374FFF0124423EF606EF439
:103C0E00606B852C82852B83E493B507EC752D01B3
:103C1E00E52C252DF582E4352BF583E49360259074
:103C2E007378E0252DFF907377E03400FE1243E9A0
:103C3E00E52C252DF582E4352BF583E493B50704A9
:103C4E00052D80CCE52C252DF582E4352BF583E46E
:103C5E009370A6E52D24FFFFE434FFFE907378E009
:103C6E002FF0907377E03EF07E007F0122E4FEFF9E
:013C7E002223
:1033DB007E147F79123BFAEF4E70037F01227E142D
:1033EB007F7C123BFAEF4E600C124423EF24D02467
:1033FB00FF920F8002D20F7E147F82123BFAEF4EA8
:10340B00600C124423EF24D090774DF08005E490AC
:10341B00774DF07E147F88123BFAEF4E600C12440E
:10342B0023EF24D0907759F08005E4907759F07E04
:10343B00147F8E123BFAEF4E600C124423EF24D014
:10344B0024FF92018002C2017E147F94123BFAEF9B
:10345B004E600C124423EF24D090737FF08005E470
:10346B0090737FF090740A63A20190774763A20177
:10347B007F0612260630013B7E147F9A123BFAEF31
:10348B004E6030120003907747EFF01200039077F5
:10349B0048EFF0120003907749EFF012000390779A
:1034AB004AEFF012000390774BEFF0120003907786
:0634BB004CEFF07F00223F
:10419300907642E0C3947C40027F0A907642E0FE30
:1041A30004F074802EF582E43473F583EFF0BF0AD4
:1041B30027907642E0FF04F074802FF582E4347395
:1041C300F583E4F0907642E0FF123C7F90764274F0
:0941D30008F0907381E004F02271
:1040EE009080007480F090740263A201F583F582D3
:1040FE0063A2017F0812260690740A63A2019080C3
:10410E008863A2017F0A1226069080927407F0A39C
:10411E0074D0F0A37406F0907414E0FF9080B1F0A8
:10412E009080E1EFF09080957455F0A3F0908000B0
:0A413E007401F090800974F0F02283
:103F0400908009E04410F09080A0E070609080A15F
:103F14007482F09080A874FFF0A3F0A3F0A3F07F64
:103F2400039080AEEFF0A374CBF09080007402F0A5
:103F34009078A71223A7000000009078A7E0908053
:103F440040F09078A8E0908041F09078A9E09080CB
:103F540042F09078AAE0908043F0A3E4F0A3F0A3A9
:0D3F6400F0A3F0908018F0A3F0A3F0A3F0FC
:013F7100222D
:10409200908009E04440F09080D17482F07F0390D8
:1040A20080DEEFF0A374CCF09080027402F090787E
:1040B200AB1223A7000000009078ABE0908058F08C
:1040C2009078ACE0908059F09078ADE090805AF012
:1040D2009078AEE090805BF0A3E4F0A3F0A3F0A3AD
:0B40E200F0908030F0A3F0A3F0A3F0FA
:0140ED0022B0
:103E8A00908009E04420F09080B8E0706C9080B98E
:103E9A007482F07F039080C6EFF07FCDA3EFF07FAE
:103EAA00039080C4EFF0A374CDF09080C074FFF04B
:103EBA00A3F0A3F0A3F09080017402F09078AF12FF
:103ECA0023A7000000009078AFE090804CF0907833
:103EDA00B0E090804DF09078B1E090804EF090780C
:103EEA00B2E090804FF0A3E4F0A3F0A3F0A3F09027
:093EFA008024F0A3F0A3F0A3F072
:013F0300229B
:103D04008C268D27A907EAFDE975F018A424ACFFD9
:103D1400E5F034808F82F583EDF0EBFDE975F01862
:103D2400A4FFAEF024ACFBEE34808B82F583A3EDCC
:103D3400F08527828C83E0FDEF24A8FFEE3480FE1B
:103D44008F82F583EDF08527828C83A3E08F828EAA
:103D540083A3F0852782852683A3A3E0FDE975F07C
:103D640018A424A8FFE5F03480FE8F82F583A3A372
:103D7400EDF08527828C83A3A3A3E08F828E83A397
:043D8400A3A3F022E3
:063AEC008D2BAB07AA06BA
:103AF200908000E030E5079076447401F0229078DF
:103B0200A7E0FCA3E0FDA3E0FEA3E0F52F8E2E8D3F
:103B12002D8C2CAE02AF038E838F8263A201E52E21
:103B2200540744C0F583852F8263A201AF2B12266E
:103B320078E4FCFDFEE52F252BF52FEE352EF52E34
:103B4200ED352DF52DEC352CF52C908040E52CF043
:103B5200A3E52DF0A3E52EF0A3E52FF090800074ED
:103B620020F0AF2FAE2EAD2DAC2C9078A712239B58
:013B72002230
:063B73008D26AB07AA0637
:103B7900908002E030E5079076447403F022907853
:103B8900ABE0FCA3E0FDA3E0FEA3E0F52A8E298DBE
:103B9900288C27AE02AF038E838F8263A201E529A9
:103BA900540744D0F583852A8263A201AF261226E1
:103BB90078E4FCFDFEE52A2526F52AEE3529F529C6
:103BC900ED3528F528EC3527F527908058E527F0BD
:103BD900A3E528F0A3E529F0A3E52AF09080027473
:103BE90020F0AF2AAE29AD28AC279078AB12239BE1
:013BF90022A9
:02372C008F27E5
:10372E00908001E030E5099076447402F07F00222B
:10373E009078AFE0FCA3E0FDA3E0FEA3E0F52B8EB6
:10374E002A8D298C2890774763A201E52A540744D5
:10375E00C8F583852B8263A2017F0612268EE52B88
:10376E002406F52BE4352AF52AE43529F529E43526
:10377E0028F52890764563A201E52A540744C8F53A
:10378E0083852B8263A201AF2712268EE4FCFDFEF9
:10379E00E52B2527F52BEE352AF52AED3529F529CA
:1037AE00EC3528F52890804CE528F0A3E529F0A308
:1037BE00E52AF0A3E52BF09080017420F0AF2BAE3C
:0D37CE002AAD29AC289078AF12239BAF27BD
:0137DB0022CB
:103106009081E0E0F52605260526052605260526F6
:1031160005260526052605260526908010E0F529B4
:10312600A3E0F52AA3E0F52BA3E0F52C9081E1E0DE
:10313600F526052605260526052605260526052641
:10314600052605260526908014E0F52DA3E0F52E2C
:10315600A3E0F52FA3E0F530E52FB52B08E530B554
:103166002C037F0022E4F526E52F540744E0F5837F
:1031760085308263A20190744163A2017F08122602
:10318600BE90744363A20190737963A2017F061215
:103196002606907441E0F527A3E0F528E4F526908D
:1031A6007441E0702AA3E024F8F526E52F5407447D
:1031B600E0F58385308274082582F582E43583F54F
:1031C6008363A20190744163A201AF261226BEAEAC
:1031D60027E4FCFDE5302528F530E52F3EF52FEDFB
:1031E600352EF52EEC352DF52D908014E52DF0A31A
:1031F600E52EF0A3E52FF0A3E530F09080007440B3
:03320600F0AF2600
:0132090022A2
:102A82009081E6E0F526052605260526052605267B
:102A920005260526052605260526908028E0F52927
:102AA200A3E0F52AA3E0F52BA3E0F52C9081E7E063
:102AB200F5260526052605260526052605260526CC
:102AC20005260526052690802CE0F52DA3E0F52E9F
:102AD200A3E0F52FA3E0F530E4F526E52FB52B0AA8
:102AE200E530B52C05C208022BEEE52F540744F061
:102AF200F58385308263A20190744163A2017F084D
:102B02001226BE907441E0F527A3E0F528E528459A
:102B12002770099080027410F07F002290774EE0B7
:102B2200FFF46030907443E06F6003022BB590773E
:102B32004FE0FF907444E06F7079907750E0FF901F
:102B42007445E06F706D907751E0FF907446E06FCE
:102B52006031805F907443E090774EF0907444E06F
:102B620090774FF0907445E0907750F0907446E083
:102B7200907751F0907447E0FFA3E0907415CFF086
:102B8200A3EFF0907441E0702AA3E024F8F526E563
:102B92002F540744F0F58385308274082582F5822C
:102BA200E43583F58363A20190744163A201AF26E9
:102BB2001226BEAE27E4FCFDE5302528F530E52FD0
:102BC2003EF52FED352EF52EEC352DF52DAF2CAE35
:102BD2002BAD2AAC29AB30AA2FA92EA82DD31223B4
:102BE2008A40099080027410F07F002290802CE5C8
:102BF2002DF0A3E52EF0A3E52FF0A3E530F09080B1
:062C0200027440F0AF2651
:012C080022A9
:102C09009081E3E0F52605260526052605260526F5
:102C19000526052605260526052690801CE0F529AA
:102C2900A3E0F52AA3E0F52BA3E0F52C9081E4E0DD
:102C3900F526052605260526052605260526052643
:102C4900052605260526908020E0F52DA3E0F52E22
:102C5900A3E0F52FA3E0F530E4F526E52FB52B0A1F
:102C6900E530B52C05C209022D5FE52F540744E86C
:102C7900F58385308263A2019070CF63A2017F0E34
:102C89001226D49070CFE0F527A3E0F5289070D7ED
:102C9900E0FFF4604A907747E0FEEF6E7079A3E0B9
:102CA900FF9070D8E06F706F907749E0FF9070D90E
:102CB900E06F706390774AE0FF9070DAE06F7057C9
:102CC90090774BE0FF9070DBE06F704B90774CE0B2
:102CD900FF9070DCE06F703FE49070DEF080089048
:102CE90070DE74FFF0D2D99070CFE0702AA3E0248F
:102CF900F2F526E52F540744E8F583853082740EF2
:102D09002582F582E43583F58363A2019070CF6350
:102D1900A201AF261226D4AE27E4FCFDE530252812
:102D2900F530E52F3EF52FED352EF52EEC352DF549
:102D39002DAF2CAE2BAD2AAC29AB30AA2FA92EA8CA
:102D49002DD312238A5006E5284527700990800162
:102D59007410F07F0022908020E52DF0A3E52EF07D
:102D6900A3E52FF0A3E530F09080017440F0AF2681
:012D79002237
:0432F3008E2C8F2D61
:1032F700908000E030E5079076447401F0229078E2
:10330700A7E0FCA3E0FDA3E0FEA3E0F5338E328D3A
:10331700318C30E533FFE5325407FEE42FF52FEE0D
:1033270034C0F52E852F82F5837423F0052FE52F02
:103337007002052E532EC7F582852E83740AF00579
:103347002FE52F7002052E532EC790740A63A20132
:10335700852E83852F8263A2017F06122678740645
:10336700252FF52FE4352EF52E852C83852D8263A9
:10337700A201852E83852F8263A20112265CE4FCBD
:10338700FDFE9078A7E0F8A3E0F9A3E0FAA3E02F09
:10339700FFEE3AFEED39FDEC38FCEF2408FFE43E82
:1033A700FEE43DFDE43CFC9078A712239B9078A7B0
:1033B700E0908040F09078A8E0908041F09078A964
:1033C700E0908042F09078AAE0908043F0908000EF
:0333D7007420F06F
:0133DA0022D0
:0A2FFF008E2B8F2C8C2D8D2E8B2F26
:10300900908000E030E5079076447401F0229078D2
:10301900A7E0FCA3E0FDA3E0FEA3E0F5358E348D27
:10302900338C32E535FFE5345407FEE42FF531EEF4
:1030390034C0F530853182F5837423F00531E531EB
:10304900700205305330C7F582853083740AF00564
:1030590031E531700205305330C790740A63A2011B
:1030690085308385318263A2017F06122678740632
:103079002531F531E43530F530852B83852C826394
:10308900A20185308385318263A20112265C8F36C5
:10309900EF2531F531E43530F530E52F6017852D11
:1030A90083852E8263A20185308385318263A201E3
:1030B900AF2F122678E5362408252FF52FFFE4FCDB
:1030C900FDFEE5352FF535EE3534F534ED3533F5BF
:1030D90033EC3532F532908040E532F0A3E533F038
:1030E900A3E534F0A3E535F09080007420F0AF3506
:0C30F900AE34AD33AC329078A712239BAC
:0131050022A7
:023C7F008F3F75
:103C8100908000E030E5079076447401F02290784E
:103C9100A7E0FCA3E0FDA3E0FEA3E0F5438E428D87
:103CA100418C40E543FFE5425407FEE42FFFEE342B
:103CB100C090738063A201F5838F8263A201AF3F3D
:103CC100122678E4FCFDFEE543253FF543EE35423F
:103CD100F542ED3541F541EC3540F540908040E548
:103CE10040F0A3E541F0A3E542F0A3E543F0908065
:103CF100007420F0AF43AE42AD41AC409078A712C2
:023D0100239B02
:013D0300229D
:0634C1008E298F2AAB05E5
:1034C700908000E030E5079076447401F022907810
:1034D700A7E0FCA3E0FDA3E0FEA3E0F5308E2F8D6F
:1034E7002E8C2DE530FFE52F5407FEE42FF52CEE4B
:1034F70034C0F52B852C82F5837423F0052CE52C3D
:103507007002052B532BC7F582852B83EBF0052C17
:10351700E52C7002052B90740A63A201852B838525
:103527002C8263A2017F061226787406252CF52CBF
:10353700E4352BF52B532BC7E529852C82852B8367
:10354700F0052CE52C7002052B532BC7F582852B34
:1035570083E52AF0052CE52C7002052B532BC7E5D4
:1035670030240AF530E4352FF52FE4352EF52EE417
:10357700352DF52D908040E52DF0A3E52EF0A3E540
:103587002FF0A3E530F09080007420F0AF30AE2F1D
:0A359700AD2EAC2D9078A712239BF7
:0135A1002207
:1043E900A2AF9210C2AF438E2075D2028F828E8304
:0C43F900E0FFE4F5D2538EDFA21092AF7B
:014405002294
:10437D00E5D220E0FBA2AF9210C2AF43D2028F82F2
:10438D008E83EDF075D25063D250A21092AFE5D26C
:03439D0020E0FB22
:0143A00022FA
:103E0C00E4FDED2401FFE433FE1243E974022DF5C9
:103E1C0082E43474F583EFF00DBD3FE6E4FDED2450
:103E2C007FFFE433FE1243E974F82DF582E434711C
:103E3C00F583EFF074F82DF582E43471F583E070BE
:103E4C001B74F82DF582E43471F5837420F074F949
:103E5C002DF582E43471F583E4F080040DBD80BE51
:103E6C00E4907277F0FDEDFF7E001243E974782D3B
:0D3E7C00F582E43472F583EFF00DBDFEE930
:013E89002216
:024299008B2B6D
:10429B00A2AF9210C2AF85A22C53A2FE8E838F8247
:1042AB0005A28C838D827409122702E52B53A2FE83
:1042BB0043A22012270453A2DF852CA2A21092AF97
:0142CB00FFF3
:0142CC0022CF
:10440600A2AF9210C2AF8C838D82EF12270243A215
:0C4416002012270453A2DFA21092AFFF77
:014422002277
:0243A1008F2665
:1043A300A2AF9210C2AFE4F5838D82740612270286
:1043B300E52643A22012270453A2DFA21092AF7F67
:0143C30001F8
:0143C40022D6
:0243C5008F2641
:1043C700A2AF9210C2AFE4F5838D82740A1227025E
:1043D700E52643A22012270453A2DFA21092AF7F43
:0143E70001D4
:0143E80022B2
:10252B00A907E7FFA805EF93C3966008403B74FC2F
:10253B002FFF80F00F08EF93C3966008402B74FBBE
:10254B002FFF80E00F08EF93C3966008401B74FACF
:10255B002FFF80D00F08EF93D3966008400B74F9D0
:10256B002FFF80C01F1F1F1F1FEF54FEF80303F721
:10257B00E893FC08E893FD08E893FE08E893FF2234
:10258B0009E993C39D6008402974FB29F980F1097F
:10259B00E993C39E6008401A74FA29F980E209E9AD
:1025AB0093D39F6008400B74F929F980D31919193B
:1025BB001919E9C313C313FF22740093F8ECC398E2
:1025CB004024701F740193F8EDC398401970147474
:0E25DB000293F8EEC398400E7009740393F853
:1025E900EFC39840037F00227F0122EDF8E6F0084F
:1025F900A3DFFA22EDF8E0F608A3DFFA22E0A363ED
:10260900A201F0A363A201DFF475A2002263A20173
:10261900F0A363A20122E0A363A201F0A363A201D4
:10262900E0A363A201F0A363A201E463A201F0A302
:1026390063A201DFE175A20022E0A363A2016DFE9E
:10264900936CFDEE058393FC158363A201DFEA75A4
:10265900A200227F00E493A363A201F00F600CA300
:10266900E583C2E3F58363A20180EA75A20022E053
:10267900A363A201F0A3E583C2E3F58363A201DFAB
:10268900EE75A20022E0A363A201F0A3E583C2E4F0
:10269900D2E3F58363A201DFEC75A20022E0A36314
:1026A900A201F0A3E58344F8C2E5F58363A201DF43
:1026B900EC75A20022E583C2E3F583E0A363A201DE
:1026C900F0A363A201DFEE75A20022E583C2E4D282
:0A26D900E3F583E0A363A201F0A380
:1026E30063A201DFEC75A20022E58344F8F583E0E1
:1026F300A363A201F0A363A201DFEE75A20022F996
:1027030022C002C004C00612FFF0D006D004D002DB
:0127130022A3
:10392F004572724C656E210A000A496E49503A0081
:10393F00205544502054696D654750530A00200AA2
:10394F00495054696D653A2000200A44415441475B
:10395F0052414D3A20002049676E6F72650A200070
:10396F002043414E2054696D654750530A0020543F
:10397F007261737353656E644552520A000ACEF832
:10398F00C4EBE8EDFB43414E210A000A4572724138
:10399F00647243414E3A00205265496E6974204368
:1039AF00414E0A002043414E283029203E20544FDB
:1039BF00210A0020545520300A0020545520310A86
:0139CF0000F7
:03001E00E4FF22DA
:10432E00C2A9438902758C48758A4875D90475DB14
:10433E004875DC4875DD4875DE48E4F5E9F5F9D2D7
:08434E00D9C2DAD28CD2DE22C2
:10430000C2D990776FE07013E5E92419F5EB30D747
:1043100006E5F904F5FB2285F9FB22E5E924C8F559
:0E432000EB30D706E5F904F5FB2285F9FB2208
:1041DC00C2D990776FE0702C301D16E5E92432F5CA
:1041EC00EB30D707E5F904F5FB800385F9FBC21D1D
:1041FC0022E5E92405F5EB30D706E5F904F5FB22B9
:10420C0085F9FB22E5E92432F5EB30D706E5F90414
:07421C00F5FB2285F9FB22EE
:1043560012432E90776FE0C394645006123D881284
:104366004300120022D21CE4F56D907887F0F55CCC
:07437600F571C21DF56F2275
:10422300EF24FCF55CD3940D4010200B077E397FFF
:104233002F1232F3E4F55CD21A2290744563A20183
:1042430090787763A201AF5C122606C21A200B0D89
:0E4253007E397F387C747D45AB5C122FFF22D4
:0F444D00D3EF6480948D5006E57170028F712259
:101C730020D903021D77201C03021D77E5716067DD
:101C83009070CF540FFF7D5E1225FDE55E640170F9
:101C93003A9070DEE0B4FF0ED21E200B127E397F25
:101CA3003F1232F38009301E06E4F571021D7712EC
:101CB3004300123F72200B0D7E397F4D7C707DCF28
:101CC300AB71122FFFE4F571021D77124300123F2F
:101CD30072200B0D7E397F587C707DCFAB71122F34
:101CE300FFE4F571021D77E55C605590787BE02495
:101CF30005F526D3940D4007E4F55CD21A80759060
:101D03007877E526540FFF7D5E1225FDE55E30E70B
:101D130002D21DE55E6401701A301E17E561B4013D
:101D230012200B127E397F657C707DCFAB71122F31
:101D3300FF8003123F72124300E4F55CD21A803431
:101D4300E56E601E90775B540FFF7D5E1225FDE507
:101D53005EB40103201E03123F72124300E4F56ECA
:101D63008012201F0C90776FE0C3946450031235E8
:101D7300A2124300122D7A8F26EF7003021EA0E4F5
:101D8300F56FE55E30E70AE561B41905D2D9021EA5
:101D9300A01241DCE55EB4010CD21E200B077E3994
:101DA3007F6F1232F3E570C394C8501B300318746D
:101DB300702570F582E43477F583E5262570F57098
:101DC3007D5EAF261225F4300121E55E20E71C90ED
:101DD30076457D5EAF261225F4AF2612372CEF70C1
:101DE3000A200B077E397F7D1232F3E55E54816052
:101DF30003021EA0E526D3940D4010300B03021EF0
:101E0300A07E397F8C1232F3021EA0E560D39407C3
:101E1300401F300B03021EA09071D07D5EAF2612CF
:101E230025F47E397F9A7C717DD0AB26122FFF80FB
:101E33006CE50F30E6629078A2E0FF90400393FEDA
:101E4300547F655E7052EFA3936560704B9078A2E8
:101E5300E0C313FF2489F582E43478F583E0703816
:101E6300530F3F9078A2E0FD7471250FF582E4349F
:101E730061F583EEF0ED90400493FE7472250FF547
:101E830082E43461F583EEF074892FF582E43478CB
:101E9300F5837401F0430F40AF26122ED5300E1A8E
:101EA30030001590776FE0C39464500C056FE56FB5
:101EB30094F04004C2AF80FEC20E200203021FB89A
:101EC300E56D6031D394014004156D8028907887C7
:101ED300E004F0E0D39403400D200B077E397FA686
:101EE3001232F3124356200B077E397FB31232F3BB
:101EF300E4F56DD21CE56E6003021FB6301B3F9004
:101F0300775B04F0A37408F0A37480F0A37401F06A
:101F1300A37406F0907872E0907760F0907873E0A5
:101F2300907761F0907874E0907762F0907875E044
:101F3300907763F0E4A3F0A3F0756E0BC21B301926
:101F430072907870E07035E56E703190775B744213
:101F5300F0A37408F0907871E090775DF090787654
:101F6300E090775EF0A37401F0756E06200B077E98
:101F7300397FC21232F3907870E004F0907870E009
:101F83006402702FE56E702B90775B7402F0A3747C
:101F930008F0907871E090775DF0A3F0A37401F0FE
:101FA300756E06200B077E397FC91232F390787065
:0A1FB300E004F0C202121FBEC200DB
:011FBD002201
:1042CD00E570602CE4907541F0A3E570F0907746B1
:1042DD00E0907543F0A37419F090777063A201908C
:1042ED00754563A201AF70122606E4F5707F0122B9
:0342FD007F00221D
:0B445C00301A05C21A7F01227F0022E7
:0100210022BC
:06448100E4F570F55C2279
:0A446700E49071D0F0A3F0A3F0225E
:103FD4002043616E457247495400200A00457272BD
:103FE4004C656E43616E21000A002043616E457288
:103FF40072434821000A205265714572722100C43F
:1040040000C401C402C403C404C405C406C407C86C
:1040140000C801C802C803C804C805C806C807C246
:1040240000C201C202C203C204C205C206C2070022
:01403400008B
:102D7A00E59B541F6020200B1A7E3F7FD41232F34A
:102D8A00E59B541FFF7E007D031234C17E3F7FDE28
:102D9A001232F3E4F59BE5BA30E010E4F5B375B10D
:102DAA0080F5B2D21CF56D907887F0E5CFF4700308
:102DBA00022ED2752801E4F527E5CFF455287003D1
:102DCA00022EC0E527C454F0F5B1E5B2547F642061
:102DDA006003022E91E5B3540FF56285BC5EE5BD32
:102DEA00541FFF131313541FFFE5BD54E044184F3B
:102DFA00F55FE5BDC43354E0FFE5BE131313541F5A
:102E0A004FF560E5BEC43354E0FFE5BF1313135416
:102E1A001F4FF56185A36385A36485A36585A366B2
:102E2A0085A36785A36885A36985A36AE4F5B220AB
:102E3A001F0FE55E547EB55E0843BDF875B350803A
:102E4A000375B3D0E562700AE55E547EB55E037F12
:102E5A000022301F08E55E30E7037F0022E562D3D7
:102E6A009408401D200B177E3F7FE11232F3AF62B8
:102E7A007E007D031234C17E3F7FEC1232F37F0065
:102E8A0022E5622405FF22E5B2549F6023200B202D
:102E9A007E3F7FEE1232F3AFB27E007D031234C161
:102EAA00AFB37E007D031234C17E3F7FEC1232F352
:102EBA00E4F5B275B3D0E52825E0F5280527E5271E
:0A2ECA00C394085003022DC37F00DB
:012ED40022DB
:103F720090776FE0C39464505675B180E4F5B3F561
:103F8200B2855EBCE560C4135407FFE55F54E04FA1
:103F9200F5BDE56033333354F8FFE561C4135407CC
:103FA2004FF5BEE56133333354F8F5BF8563A3851E
:103FB20064A38565A38566A38567A38568A38569D0
:103FC200A3856AA3E562540F2450F5B3756D0AC246
:023FD2001C22AF
:1035A20075B190E5B220E613200B107E3F7FF91231
:1035B20032F3AFB27E007D031234C1E4F5B3F5B24B
:1035C200E50F30E615E4F50F9078A2E02402F0E072
:1035D2009040039370049078A2F07471250FF582E5
:1035E200E43461F583E0702D9078A2E0FFC31324E8
:1035F20089F582E43478F583E07005430F80801505
:10360200E4F50F9078A2E02402F0E090400393707A
:10361200049078A2F0E50F30E7219078A2E0FF90C5
:10362200400393F5BCE4F5BDEFA393FF333333546A
:10363200F8F5BE75BF78430F4080367471250FF5DB
:1036420082E43461F583E0F5BC75BD807472250FA8
:10365200F582E43461F583E0FF33333354F8F5BE89
:1036620075BF78050F050FE50FC394324003E4F5EB
:053672000F75B35022AA
:09447100EF6003C29622D29622EC
:103D880043AB01C2E8C2EAE4FFEFC454F0F5B1C3A3
:103D9800EF64809488500575B3D08003E4F5B3E4EC
:103DA800F5B2F5BCF5BDF5BEF5BFF5C4F5C5F5C66C
:103DB800F5C7F5A3F5A3F5A3F5A3F5A3F5A3F5A317
:103DC800F5A30FBF0EC390776FE0FE25E0F5B4753D
:103DD800B50C75B66C75A11275AB0275C13E75C38D
:103DE800FF75C203E49078A2F0750F80FF7F1990E9
:103DF8007889E4F0A3DFFCE4FF7F32906171E4F09E
:033E0800A3DFFC39
:013E0B002294
:1014A0003E2A2C312CCFE0F0E0ECE5F2F0FB20F30B
:1014B000EFF0E0E2EBFFFEF9E5E3EE20EAEEEDF21D
:1014C000F0EEEBEBE5F0E020CACF20C8F1E5F2FC4E
:1014D0000A003E4C2C6B30312C25732C43EAEEF085
:1014E000EEF1F2FC20EDE020F8E8EDE52043414E7E
:1014F0002C30202D20353030EAE1283530EC292CF5
:1015000031202D203530EAE128353030EC290A0031
:1015100030202D20353030EAE1283530EC290031FB
:10152000202D203530EAE128353030EC29003E42CC
:101530002C6330312C2562752CC2F2EEF0E8F7ED09
:10154000FBE920EAEEEDF2F0EEEBEBE5F020EDE06A
:1015500020F8E8EDE50A003E2A2C312CCFF0EEF21F
:10156000EEEAEEEB20C8F1E5F2FC2DCCE0E3E8F189
:10157000F2F0E0EBFCEDFBE920EDE020EFEEF0F225
:10158000F32052533233320A003E4C2C6B30352C50
:10159000256C752CD1EAEEF0EEF1F2FC20EEE1ECD8
:1015A000E5EDE020EDE020EFEEF0F2F32C3130300D
:1015B0002C3230302C3330302C3630302C3132302D
:1015C000302C323430302C343830302C3936303006
:1015D0002C31393230302C33383430302C353736EA
:1015E00030302C3131353230300A003E532C6B30E4
:1015F000362C2562752CC0E4F0E5F120CACF20E43A
:10160000EBFF20ECE0E3E8F1F2F0E0EBE80A003E6B
:10161000532C6B31332C2562752CC7E0E4E5F0E6E2
:10162000EAE020F1F2E0F0F2E020EFE5F0E5E4E0BE
:10163000F7E828E1E0E9F2290A003E422C6B31305C
:101640002C2562752CCFE5F0E5E7E0E3F0F3E7EA5F
:10165000E020EFF0E820EEF2F1F3F2F1F2E2E8E858
:1016600020EEE1ECE5EDE0203220ECE8ED2E0A0082
:101670003C21003C6B30313D003C6330313D003C4F
:101680006B30353D003C6B30363D003C6B31333DBB
:10169000003C6B30393D003C6B31303D00545520EF
:1016A0005265710A005455204F4B0A00CEF820E4D1
:1016B000EBE8EDFB210A000A4173796E634F555444
:1016C0003A002054552054696D65210A000A43529E
:1016D00043204552523A20000A4173796E63494EC5
:1016E0003A00CFE0EAE5F220E22043414E0A000A48
:1016F000CFF0E8EDFFF2E020EAEEECE0EDE4E020F0
:10170000D2D320002020D2D320E7E0EDFFF2EE215B
:101710000A003F3F3F0A000089129B24AD36BF48B4
:10172000C15AD36CE57EF78108931AA52CB73EC940
:1017300040DB52ED64FF76028B109926AF34BD4A30
:10174000C358D16EE77CF5830A9118A72EB53CCB20
:1017500042D950EF66FD74048D169F20A932BB4C10
:10176000C55ED768E17AF3850C971EA128B33ACD00
:1017700044DF56E960FB72068F149D22AB30B94EF0
:10178000C75CD56AE378F1870E951CA32AB138CFE0
:1017900046DD54EB62F97008811A932CA53EB740E0
:1017A000C952DB64ED76FF89009B12AD24BF36C1C0
:1017B00048D35AE56CF77E0A8318912EA73CB542B0
:1017C000CB50D966EF74FD8B029910AF26BD34C3A0
:1017D0004AD158E76EF57C0C851E9728A13AB34490
:1017E000CD56DF60E972FB8D049F16A920BB32C580
:1017F0004CD75EE168F37A0E871C952AA338B14670
:10180000CF54DD62EB70F98F069D14AB22B930C75F
:101810004ED55CE36AF17800112332465765748C2B
:101820009DAFBECADBE9F810013322564775649CB0
:101830008DBFAEDACBF9E82130021367764455AD9F
:10184000BC8E9FEBFAC8D93120120377665445BD90
:10185000AC9E8FFBEAD8C94253617004152736CE7F
:10186000DFEDFC8899ABBA5243716014053726DE70
:10187000CFFDEC9889BBAA6372405125340617EF5F
:10188000FECCDDA9B88A9B7362504135241607FF50
:10189000EEDCCDB9A89A8B8495A7B6C2D3E1F00847
:1018A000192B3A4E5F6D7C9485B7A6D2C3F1E01830
:1018B000093B2A5E4F7D6CA5B48697E3F2C0D1291F
:1018C000380A1B6F7E4C5DB5A49687F3E2D0C13910
:1018D000281A0B7F6E5C4DC6D7E5F48091A3B24AFF
:1018E0005B69780C1D2F3ED6C7F5E49081B3A25AF0
:1018F0004B79681C0D3F2EE7F6C4D5A1B082936BDF
:101900007A48592D3C0E1FF7E6D4C5B1A092837BCF
:071910006A58493D2C1E0F2F
:030023000236772B
:0D367700C0E0C0F0C083C082C0D075D01884
:1036840030985AC298750B01AF99202013BF550981
:10369400754D00D220D2918044906B88EFF0803D2C
:1036A400E55670347489254DF582E4346BF583EF67
:1036B400F0E54DB40104EF04F546E54D600AB54666
:1036C4001304F556C291800CEF64556007C2209034
:1036D4006B88EFF0054D8005906B88EFF030993DD5
:1036E400302138D290E554700DE54A6549600705EC
:1036F4004A75990A8025E554B54C10C221754A00D3
:10370400D223C290E4FF124471801074892554F5C9
:0D37140082E4346CF583E0F5990554C29908
:0B372100D0D0D082D083D0F0D0E032B6
:10388A007BFF7A1479A012197990776FE07014751A
:10389A002EFF752F157530107BFF7A1479D2121905
:1038AA00798012752EFF752F1575301F7BFF7A14DC
:1038BA0079D21219797BFF7A15792EA21FE433F592
:1038CA002E1219797BFF7A1579571219799070C9D6
:1038DA00E0FEA3E0FFC3E49FFFE49EFEAB07FA33DA
:1038EA0095E0F9F87F007E8C7D0A7C001222EA8F2F
:1038FA00318E308D2F8C2E7BFF7A157989121979AA
:10390A007BFF7A1579EB85552E1219797BFF7A168A
:10391A00790F85492E1219797BFF7A16793A8557DC
:05392A002E12197922A4
:10320A007E167F70123BFAEF4E70037F0122E49024
:10321A00776FF07E167F73123BFAEF4E60151244F9
:10322A0023BF310690776F740AF0BF320690776F2A
:10323A007464F07E167F79123BFAEF4E600D1240ED
:10324A0035EC4D4E4F24FF921F8002C21F7E167F1F
:10325A007F123BFAEF4E6023124035A804A905AA53
:10326A0006AB077F007E8C7D0A7C001222EA1223BD
:10327A007C9070C9EEF0A3EFF0800A9070C974FFD9
:10328A00F0A374B8F07E167F85123BFAEF4E600702
:10329A001240358F558003755501906B867401F085
:1032AA007E167F8B123BFAEF4E60071240358F492C
:1032BA008003E4F5497E167F91123BFAEF4E600CCB
:1032CA00124423EF24D024FF92228002D2227E16B7
:1032DA007F97123BFAEF4E600A124423EF24D0F58F
:0832EA00578003E4F5577F0053
:0132F20022B9
:1037DC00C221C223C220E4906B87F0F554F54CF55E
:1037EC00089061A4F0F54DF50BF54A9070C974FF83
:1037FC00F0A374F4F012320AE4F50FF558E558759D
:10380C00F00DA42403F582E43461F583E4F0F54B68
:10381C0075F068E558A42489F582E5F0346DF583DC
:10382C0075F00DE54B1223D8E4F0054BE54BB408CD
:10383C00DF0558E558B408C5E4F55BF544F545F5E6
:10384C0047F553F558F54BF552C2ADF5C9D2CDD26B
:10385C00CCC2C9C2CAF5CDF5CC9070C9E0F5CBA3EA
:10386C00E0F5CA85CBCD85CACCD29ED29CD2CAC239
:0E387C00ACC298C29975B81075B710D2AC22C4
:0100220022BB
:102ED5008F27E55EB44209E56164027003022FFEA7
:102EE500E55F54E324DF607824DF7003022FBA1412
:102EF5007003022FCE24E37003022F8D147003029A
:102F05002F8D24E1601E24606003022FFEE56075AD
:102F1500F00DA42403F582E43461F5837D5EAF27CB
:102F25001225F422E56075F00DA42403F582E4343E
:102F350061F583E4F075F00DE547A42446F582E5D7
:102F4500F03468F5837D5EAF271225F405475347B6
:102F55003FE54565476003022FFE054553453F2282
:102F650075F00DE544A424C5F582E5F03461F583DB
:102F75007D5EAF271225F4054453447FE544655B28
:102F85007077055B535B7F22435F0143618075F07A
:102F950068E560A42489F582E5F0346DF583E56183
:102FA500543FFF1313543F75F00D1223D87D5E7FF8
:102FB5000D1225F422300C077E167F9D1232F33058
:102FC50019379078707402F022300C077E167FA5B1
:102FD5001232F375F00DE547A42446F582E5F03489
:102FE50068F5837D5EAF271225F4054753473FE516
:0A2FF50045B54705054553453F2249
:104148008E2A8F2B8F828E83E5822404F582E435B4
:1041580083F583E02405F554D3940E400B200B2AF5
:104168007E167FAC1232F322852A83852B8263A2C6
:104178000174892552F582E4346CF58363A201AF9A
:0B41880054122606E5542552F5522281
:10271400E4F529755206F528906B86E0FFE529C398
:102724009F400302284EE5476545601E75F00DE5A0
:1027340045A42446F582E5F03468AF82FE12414890
:102744000529054553453F022842E54814602E14E7
:1027540060728000E4F548E544655B601E75F00D29
:10276400E55BA424C5F582E5F03461AF82FE124135
:10277400480529055B535B7F0228420548E55375EC
:10278400F00DA42403F582E43461F583E0602EE5C2
:102794005375F00DA42403F582E43461AF82FE1274
:1027A4004148E55375F00DA42403F582E43461F542
:1027B40083E4F00553535307052902284205535374
:1027C4005307054875F068E558A42489F582E5F0B7
:1027D400346DF58375F00DE54B1223D8E0604C752C
:1027E400F068E558A42489F582E5F0346DF5837525
:1027F400F00DE54B1223D8AF82AE8312414875F039
:1028040068E558A42489F582E5F0346DF58375F004
:102814000DE54B1223D8E4F0E54BC394084008E4DB
:10282400F54B055853580705298013054BE54BC351
:1028340094084008E4F54B05585358070548052803
:10284400E528C3940A500302271CE55224FAF5290B
:10285400906C897455F0A3F0E5292405A3F0E4A352
:10286400F0A3E555F0906845E0906C8EF0E4F54EE9
:10287400F54FE5292403F551906C8C63A201901760
:102884001763A201AF51AE50AD4FAC4E1226428F2A
:10289400518E508D4F8C4E748F2529F582E4346C03
:1028A400F583E54FF074902529F582E4346CF583C3
:1028B400E54EF0E5292408F54CD221E4F554906165
:1028C4006FF07F01124471D299200B0D7E167FB7F1
:0928D4007C6C7D89AB4C122FFFD6
:0128DD0022D8
:101FBE00E55375F00DA42403F582E43461F583E056
:101FCE007005055353530775F068E558A42489F539
:101FDE0082E5F0346DF58375F00DE54B1223D8E0F4
:101FEE007011054BE54BC394084008E4F54B0558BA
:101FFE00535807300034C20030191890616EE00457
:10200E00F0E0D3940A400C200B077E167FC21232EA
:10201E00F3C219E557600D0557E557D394F0400408
:10202E00C2AF80FE90616FE004F030DA3FC2DA900A
:10203E0061A4E0FF906B87E0FDC39F502FE55A250A
:10204E00ECF5EC30D709E55925FC04F5FC8006E5E6
:10205E005925FCF5FC74A52DF582E43461F583E079
:10206E00B55503122714906B87E004F030210F90C2
:10207E00616FE0D39414400BC221D2238005E4900B
:10208E00616FF0906B88E0FF600C7E007D03123470
:10209E00C1E4906B88F0E55670030222ADF527E49B
:1020AE00F54EF54FE52724FEF551906B8B63A2019B
:1020BE0090171763A201AF51AE50AD4FAC4E122622
:1020CE00428F518E508D4F8C4EC220E4F556E54F07
:1020DE00454E601D300B030222AD7E167FCD7C6B0C
:1020EE007D89AB27122FFF7D03AF4FAE4E1234C149
:1020FE0022200B0D7E167FD87C6B7D89AB27122F8D
:10210E00FFE5576003755701906B8BE0FB64016030
:10211E0003022202906B8DE09061A3F06007E02035
:10212E00E7030222AD9061A3E0547FF0906845F082
:10213E00E5E92402F5EC30D707E5F904F5FC800358
:10214E0085F9FCC2DA906B8CE075F064A485F059C9
:10215E00F55A906B8EE0FE541F9061A4F0EEC413FE
:10216E00540704906B86F0E4A3F0F5279061A4E089
:10217E00FFE527C39F501E748F2527F582E4346B2D
:10218E00F583E0FF74A52527F582E43461F583EF2E
:10219E00F0052780D7748F2527F582E4346BF583FD
:1021AE00E0F460030222AD74912527F582E4346BCE
:1021BE00F583E0FF907873E06F70030222AD7490A8
:1021CE002527F582E4346BF583E0907872F0A3EF67
:1021DE00F074922527F582E4346BF583E0907874E1
:1021EE00F074932527F582E4346BF583E0907875CF
:1021FE00F0D21B22906B8CE0655560030222ADEB92
:10220E0024FD604E0460030222A3200B077E167F7E
:10221E00E21232F3E56E60030222AD756E0D906B25
:10222E008E63A20190775B63A201AF6E12260690B9
:10223E00775BE0FFB4440B907760E0B40104E4F503
:10224E006E22EF64447058907760E07052F545F559
:10225E004722200B077E167FEF1232F330190B2028
:10226E000B3D7E177F041232F322906B8FE0907835
:10227E0071F0906B90E025E0907876F0906B91E0A5
:10228E0020E006907876E004F0D219E490616EF0CA
:0F229E00907870F022200B077E177F121232F318
:0122AD00220E
:103A6C00020911E493A3F8E493A34003F68001F256
:103A7C0008DFF48029E493A3F85407240CC8C3335B
:103A8C00C4540F4420C8834004F456800146F6DF2A
:103A9C00E4800B010204081020408090447AE47EFC
:103AAC00019360BCA3FF543F30E509541FFEE4931F
:103ABC00A360010ECF54C025E060A840B8E493A3E6
:103ACC00FAE493A3F8E493A3C8C582C8CAC583CA11
:103ADC00F0A3C8C582C8CAC583CADFE9DEE780BEC9
:01448000003B
:1022AE0075F008758200EF2FFFEE33FECD33CDCCE7
:1022BE0033CCC58233C5829BED9AEC99E58298406A
:1022CE000CF582EE9BFEED9AFDEC99FC0FD5F0D647
:1022DE00E4CEFBE4CDFAE4CCF9A88222B800C1B971
:1022EE000059BA002DEC8BF084CFCECDFCE5F0CBAF
:1022FE00F97818EF2FFFEE33FEED33FDEC33FCEBE8
:10230E0033FB10D703994004EB99FB0FD8E5E4F9A2
:10231E00FA227818EF2FFFEE33FEED33FDEC33FC8F
:10232E00C933C910D7059BE99A4007EC9BFCE99A83
:10233E00F90FD8E0E4C9FAE4CCFB2275F010EF2FC8
:10234E00FFEE33FEED33FDCC33CCC833C810D707C8
:10235E009BEC9AE899400AED9BFDEC9AFCE899F803
:0E236E000FD5F0DAE4CDFBE4CCFAE4C8F92296
:0E237C00C3E49FFFE49EFEE49DFDE49CFC2272
:10238A00EB9FF5F0EA9E42F0E99D42F0E89C45F0A9
:01239A002220
:0C239B00ECF0A3EDF0A3EEF0A3EFF022B5
:1023A700A8828583F0D083D0821223BE1223BE1267
:1023B70023BE1223BEE473E493A3C583C5F0C5838C
:1023C700C8C582C8F0A3C583C5F0C583C8C582C880
:0123D70022E3
:0C23D800A42582F582E5F03583F5832210
:10191700E53A242EF8E6053A22782B301702782E7E
:10192700E475F00112248B0223E42010EB7F2ED202
:10193700108018EF540F2490D43440D4FF30140B88
:10194700EF24BFB41A0050032461FFE53B60021582
:101957003B053EE53E7002053D30170D782BE475DB
:10196700F00112248BEF02242A0241937403D21749
:101977008003E4C217F53A8B2B8A2C892DE4F53BBB
:10198700F53DF53EE53B60077F2012195280F5755E
:101997003CFFC211C210C212C213C215C216C2182E
:1019A700121920FF700D3017057F00121963AF3E23
:1019B700AE3D22B4255FC2D5C214121920FF24D030
:1019C700B40A00501A75F00A783B30D50508B6FFFF
:1019D7000106C6A426F620D5047002D21380D924A6
:1019E700CFB41A00EF5004C2E5D214021B63D21120
:1019F70080C6D21080C0D21280BCD2D580BAD21590
:101A070080B47F201219522012077401B53B0040A1
:101A1700F1121917FF12195202198BD218D2168018
:101A270095121917FB121917FA121917F94A4B7061
:101A37000679347A1C7BFF20122EE53B602A7E0054
:101A47008E827583001223FD60060EEE653C70F0F2
:101A5700C2D5EBC0E0EAC0E0E9C0E0EE121BAAD0B5
:101A6700E0F9D0E0FAD0E0FB1223E4FF60AAEBC074
:101A7700E0EAC0E0E9C0E0121952D0E02401F9D051
:101A8700E03400FAD0E0FBE53C0460DCD53CD980CB
:101A9700877BFF7A1B79A6D212809C791080027906
:101AA70008C216C2188008D2D5790A8004790AC2FA
:101AB700D5E53C047002F53CE4FAFDFEFF12191768
:101AC700FC7B08201113121917FD7B1030100A1226
:101AD7001917FE121917FF7B20EC3382D592D550C8
:101AE70013C3E43010069FFFE49EFEE42011039D1C
:101AF700FDE49CFCE4CBF8C211EC700CCFCECDCC4E
:101B0700E824F8F870F38017C3EF33FFEE33FEEDE8
:101B170033FDEC33FCEB33FB994002FB0FD8E9EBC9
:101B2700301105F8D0E0C448B211C0E00AEC4D4EC0
:101B37004F78207B0070C2EAB53C0040BCC0E01281
:101B47001BACD0F0D0E0201104C4C0E0C4B211C077
:101B5700F012193BD0F0D5F0EB02198B1224EA1AD8
:101B670028531AA25819F94C19F5421AA64F1AAE5A
:0F1B7700441AAE491A0E431AB4551A98461A98D2
:101B8600451A98471C545019FD2D1A012E1A242B5C
:101B96001A05231A22201C3D2A19BD4800001A1CCA
:101BA6003F3F3F00790AA2D5201314301509B9101A
:101BB600020404B9080104A2D5201602500104202B
:101BC60012689212B53B005034C0E07F20301319E2
:101BD6007F30A21272167215500F121C03C212C267
:101BE60016C215C2187F30800F301503E9C0E01207
:101BF6001952301503D0E0F9D0E0B53BCC301517BB
:101C06007F30B9100C1219527F583014077F788034
:101C160003B908031219523012057F2D0219527F9B
:101C2600202018F87F2B2016F322921280CF286EE0
:101C3600756C6C2900D2111219173011F8C211787F
:101C46003B30D50108F60219BD2D504349581219EB
:101C5600172403B405004001E4901C4F9312194366
:0D1C6600743A121943D213753B04021AA2FE
:1028DE008B268A278928E4F532F531F530F52FF568
:1028EE002DF52EE52A452B45296012EBC0E0EAC0F6
:1028FE00E0E9C0E0AB29AA2AA92B12249BAB26053E
:10290E0028E528AA277002052714F91223E4F533C7
:10291E00C394094007E533D3940D40E1E5336420B9
:10292E0060DBE533B42D05432E038016E533B42B5F
:10293E0005432E01800C74FF2528F52874FF3527DA
:10294E00F527E52C60046410703FAB26AA27A92852
:10295E001223E464306009E52C702E752C0A802950
:10296E009000011223FDFF64786004EFB458134306
:10297E002E01752C1074022528F528E43527F5272D
:10298E008007E52C7003752C08AB260528E528AAD0
:10299E00277002052714F91223E4F533C39461401E
:1029AE000AE533D3947A50035333DF74D02533F5CD
:1029BE0033C3940A400CE5339411406D74F92533FA
:1029CE00F533E533D3952C5060432E018532378590
:1029DE003136853035852F34AF2C7E00E4FCFDABCF
:1029EE0032AA31A930A82F12243CC8ECC8C9EDC9AF
:1029FE00CAEECACBEFCBE4FCFDFEEB2533F532EE8F
:102A0E003AF531ED39F530EC38F52FAF32AE31AD58
:102A1E0030FCAB37AA36A935A834D312238A50031B
:102A2E00022997432E04022997E52E20E003E48025
:102A3E002DE52A452B4529601EAB26E52824FFF9F6
:102A4E00E52734FFFAEBC0E0EAC0E0E9C0E0AB29CD
:102A5E00AA2AA92B12249BE52E30E20774FFFFFE53
:102A6E00FDFC22E52EAF32AE31AD30AC2F30E1039E
:042A7E0002237C2291
:1023E400BB010689828A83E0225002E722BBFE02F7
:0923F400E32289828A83E493222A
:1023FD00BB010CE58229F582E5833AF583E0225095
:10240D0006E92582F8E622BBFE06E92582F8E222DE
:0D241D00E58229F582E5833AF583E49322F8
:10242A00BB010689828A83F0225002F722BBFE0191
:02243A00F3228B
:10243C00E88FF0A4CC8BF0A42CFCE98EF0A42CFC3F
:10244C008AF0EDA42CFCEA8EF0A4CDA8F08BF0A4BD
:10245C002DCC3825F0FDE98FF0A42CCD35F0FCEB1C
:10246C008EF0A4FEA9F0EB8FF0A4CFC5F02ECD39E1
:0F247C00FEE43CFCEAA42DCE35F0FDE43CFC224E
:10248B00FAE6FB0808E6F925F0F618E6CA3AF62252
:10249B00BB011A89828A83D0F0D0E0F8D0E0F9D062
:1024AB00E0FAD0E0FBE8C0E0C0F00225195016E9D5
:1024BB00F8D083D082D0E0F9D0E0FAD0E0FBC08234
:1024CB00C083022510BBFE16E9F8D083D082D0E082
:0F24DB00F9D0E0FAD0E0FBC082C08302252222B4
:1024EA00D083D082F8E4937012740193700DA3A381
:1024FA0093F8740193F5828883E473740293686095
:06250A00EFA3A3A380DF94
:09251000EBF608EAF608E9F622F0
:09251900EBF0A3EAF0A3E9F022C3
:09252200EBF208EAF208E9F222EA
:00000001FF
